:020000020000FC
:10000000BACDAEC10000000020C0000093C00000C7
:1000100000009DC000000000000000000203040674
:10002000080C10182030406080000406080C1018DE
:100030002030406080A0C00000070F1F3F000D0D62
:1000400004050D050305030302004FB662FD0EC053
:10005000552009F00994C52DC095089483FDC795D6
:10006000C4BDC093A10064604FBE1895C0916400E8
:10007000089483FDC795C4BDC093A1006B7FC09158
:100080006400CF3F09F41FC070FF02C082FD05C0AD
:100090004FBEC098C198C2981895C098C198C29890
:1000A00075FD0DC065FD0BC0C9E0CA95F1F7C091A3
:1000B000B300C0FD939AC1FD949AC2FD959A209217
:1000C000A1004FBE189524BCCC27C064C8BF646093
:1000D000F6CFC1CF70FFBFCF65FDBDCFC09ABBCFFC
:1000E00070FFB9CF65FDB7CFC19AB5CF70FFB3CF61
:1000F00065FDB1CFC29AAFCF939870FFACCF65FDCD
:10010000AACFC7E0CA95F1F7C09AA5CF949870FF1F
:10011000A2CF65FDA0CFC7E0CA95F1F7C19A9BCFEA
:10012000959870FF98CF65FD96CFC7E0CA95F1F717
:10013000C29A91CF4FB6C9B7CF7EC9BF6E7FCCB53B
:10014000CE0DDDB5DF1DDBBDCABD4FBE18953FB678
:100150008F7EABB7A074A2118061A0E0ABBFA9B73E
:10016000AE7FA9BF7894A0916800AA2341F085FDD5
:100170002AC0A0916800AA95A093680024C040E01E
:1001800050E085FD14C0A0B396FDA095A2FD4FEFF1
:10019000A3E096FDA2E0A5BFAA27A064AABF8D7F19
:1001A000A0B396FDA095A2FD5FEF451741F7A8E12A
:1001B00061FDA093680085FD03C0A8E1A0936800DD
:1001C00040939700816085FD0EC0A0916900AA232D
:1001D00031F0A0916900AA95A093690004C08061E4
:1001E000AA27A064AABF80FF37C0A09197004A2F1A
:1001F00061FF8E7F85FD1CC0A091B600A430C1F4C4
:10020000403F08F040EFA42FA295AF704A0F5091E5
:10021000B800533069F0A695A69550FD01C0A6958B
:1002200052FD03C0A41B4A2F03C04A0F08F44FEF2E
:1002300040936100A72FA67079F0A0916D00A6955C
:10024000A69556E0A50F50916100A50FA0936100FF
:1002500018F4AFEFA09361004091B600443009F06C
:100260003EC0A0916100A093630040916300A09103
:100270009C004A1708F04A2FA0919E004A1708F0E8
:100280004A2F542EA091A200AA2309F422C0542F71
:100290005A1B10F4A42F50E0BA2E8894AA1FAA2E3D
:1002A000A091A400A095AA22A50E58F0A091A300A9
:1002B000A21509F0AA95AA0EA093A30048F04A2D12
:1002C00008C0A091A300BA1608F0A395A093A300BC
:1002D0004FEF409364007F7D485F08F07062A52D6A
:1002E000A03408F06860A0916000A395A09360001E
:1002F00051F0F894A9B7A160A9BF84FF02C0A0E49F
:10030000ABBF3FBE1895A0917400A395A093740055
:1003100041E050916800552329F085FF03C05A95AC
:1003200050936800A0919700A13018F020929A0095
:100330000DC020929B002092A500A0919A00AF5F73
:10034000A0939A0018F0AFEFA0939A00F894A9B781
:10035000A160A9BF84FF02C0A0E4ABBF3FBE189557
:100360003FB64CB55DB58F7EABB7A074A21180616E
:10037000A0E0ABBFA9B7AE7FA9BF789481FD23C031
:10038000A2E096FDA3E0A5BF8260A0B396FDA09574
:10039000A2FF05C040936500509366003EC1A3E0F4
:1003A00096FDA2E0A5BFAA27A064AABF8D7F85FF06
:1003B00001C026C140E0A0B396FDA095A2FD20C1DA
:1003C000409397000FC1A3E096FDA2E0A5BF8D7FEB
:1003D00061FF71C0A2E096FDA3E0A5BFAA27A064BB
:1003E000AABF82604093920050939300A090900027
:1003F0004A19B09091005B09BB24A22C4C385205DD
:1004000018F42092960049C0A091D600AA2359F171
:10041000483C520528F4A0E1BA2EAAE0AA2E23C037
:100420004836A1E05A0728F4A8E0BA2EAFE0AA2E79
:100430001AC0403DA2E05A0728F4A4E0BA2EAEE16B
:10044000AA2E11C0403AA5E05A0728F4A2E0BA2E1D
:10045000ACE3AA2E08C04839A8E05A0720F4A1E06E
:10046000BA2EA8E7AA2EC42EA0919400CA1AD52E9F
:10047000A0919500DA0ADD202AF4AFEFC094D09461
:10048000CA1ADA0A20929600A8E0A210A0E0CA14C4
:10049000DA0618F4A1E0A0939600409394005093DC
:1004A000950040919200509193004093900050939A
:1004B000910002E097C0A09165004A1BA0916600E0
:1004C0005A0B94FD82C093FD80C092FD7CC086FFD4
:1004D00003C0D52EC42E0CC05695479591FD73C010
:1004E0005695479590FD6FC0D52EC42ED694C794CF
:1004F00061FD19C0AC2DAC51AD2DA24008F005C076
:10050000DD2089F4AC2DA85C70F4A0916700A39560
:10051000AA2311F0A0936700AA3008F471C02092BA
:10052000970081606DC0A0916700AA2319F0AA9579
:10053000A0936700A22C5091BC0097FD06C0A0902C
:10054000CA00533011F4A090D200AAEFAA0EA22D37
:10055000A21DCA18DA0A4FB74170533049F4442338
:1005600021F087FD05C0806803C087FF01C08F7739
:10057000442359F0533031F4AFEFC094D094CA1AE9
:10058000DA0A03C040E050E020C0533049F4CC0CFC
:10059000DD1CAAE0CA1AD20818F4A0E0CA2ED22C98
:1005A000AFEFCA16D20418F04FEF50E00EC0A09182
:1005B000AE00CA9E412D000C441F50E008F012C04E
:1005C0004FEF50E00FC05695479594FF07C0552355
:1005D00009F04FEFA42FA6954A0F521D4F3F520529
:1005E00008F04FEF40939700816061FF09C0AFE1D1
:1005F000A095A923AB299A2F8F7DBB2009F4806297
:10060000A8E1A093680085FF03C0AAE0A09368005A
:1006100061FD03C085FD01C08F7E85FD03C0A6E09E
:10062000A0936900F894A9B7A160A9BF84FF02C094
:10063000A0E4ABBF3FBE189511E00AC013E008C0AC
:100640001AE006C01EE104C014E602C018EC00C0A7
:1006500005E1BB27BA95F1F70A95D9F71A95C1F7C5
:1006600008952AE338E709C020E33CE806C02AE2FF
:1006700034EB03C025E238EC00C012E095FD9F7D0D
:1006800095FF9062BB279498BA95F1F7C19ABA95F5
:10069000F1F7C198BA95F1F7949ABA95F1F7C09A23
:1006A000B091AF00BA95F1F7C098B7E8BA95F1F7F5
:1006B0001A9521F7022FB22FBA95F1F70A95D9F7BB
:1006C0003A95D9F694980895221B39E0001F3A957F
:1006D00009F40895221F211B18F4210F8894F6CFE6
:1006E0000894F4CF622C722CB0E08894B395221F4A
:1006F000331FE0F7379527958894912E802E020BB3
:10070000130B10F4192D082D10F4889401C00894CF
:10071000661C771CBA9571F7172D062D0895322D9A
:1007200011232AF43A9500951095031B130BF894A6
:10073000029F712C002D129F912C802C7894780CA4
:10074000172D921C292DB4E06B2E26951795079531
:100750006A94D9F7332321F000951095031B130BEE
:1007600008950091B6000430A1F1B0919700B15006
:1007700008F010C0B0916100B093630020927F0038
:10078000209280002092810020928200209283009B
:100790006F7B1FC06090B6006064B0916100B09341
:1007A000620008E317EC20917A0030917B003695C7
:1007B0002795B62DBA9541F036952795B62DBA9561
:1007C000BA9511F0369527958DDF00937F00109331
:1007D0008000089500917F00B09162000B1B109182
:1007E0008000120928F40038BFEF1B0740F009C051
:1007F0000F37120508F405C00FE710E002C000E84B
:100800001FEF0093840010938500089500918400E9
:10081000B09181000B0F10918500B09182001B1FD9
:1008200020E03091850033230AF42A95B0918300AB
:100830002B1F1AF4203F40F00AC02F3008F407C0E5
:100840000FEF1FEF2FE003C000E010E020EF30912A
:100850006300B0919C003B1718F4323030F009C0AF
:10086000B0918500BB235AF004C0B0918500BB2332
:1008700032F4009381001093820020938300089546
:100880002091D80000918400000F10918500111F65
:1008900046DF11232AF40038BFEF1B0740F009C0E0
:1008A0000F37120508F405C00FE710E002C000E89A
:1008B0001FEF002352F0B0916200B01B0B2F18F015
:1008C000013008F00AC001E008C000950F5FB09148
:1008D00062000B0F08F001C00FEF0093860008952F
:1008E0002091D900009182001091830018DF11231C
:1008F0002AF40130BFEF1B0740F009C00F3F12057B
:1009000008F405C00FEF10E002C001E01FEF112353
:1009100052F0B0918600B01B0B2F18F0013008F098
:100920000AC001E008C000950F5FB09186000B0F70
:1009300008F001C00FEF0093630008950FEF677F89
:1009400071FD29C072FD09C06860B0917B00BA30AA
:1009500020F0B52DB03408F4677FB091D500BB23EB
:10096000D1F0B0917B00BB23B1F00FEF10917B0071
:10097000ABDEF894B091730072FDB5E00B9F112DC2
:10098000002D7894112309F00FEFB0919F000B1701
:1009900010F400919F0000939E00089500917A004A
:1009A00010917B0000541140B0919E0010F4BA9554
:1009B00001C0B39511F0B0939E00089500C0089552
:1009C0002091B700B6B1B6FDFBCF04B115B1B6B1F9
:1009D000BF77B6B9B091AC00B395B093AC00B83066
:1009E00060F12092AC00B091D400BB2321F111231F
:1009F00029F0B091AD00BF3F61F009C0B091AD00EA
:100A00000B1739F020F4BB2321F0BA9502C0B3953F
:100A1000E1F300919C00B093AD00BA3F50F400ECBC
:100A2000B93F38F400E8B83F20F400E4B73F08F4D9
:100A300000E000939C00777F089510919C00B0E146
:100A40001B0F08F41FEF10939C00B091B600B43058
:100A500081F000919C00B0916300B01B10F40091F4
:100A60006300B0919E000B1708F00B2F502E0093DF
:100A70006400B091AC00B73009F47860089502E3E7
:100A8000F894B091DA000B9F012D000C001F7894B0
:100A9000B0919C000B1710F000919C000093610036
:100AA00000936300502E0093640000939F0008950C
:100AB00020927A00B0EFB0937B000895F8940CB5C3
:100AC0001DB5209174007894309175006090760087
:100AD0000093750010937600031B160971FD03C087
:100AE00076FD81C02BC07090770020937700270996
:100AF000222311F00FEF1FEF809078009090790083
:100B000030937800609279006918161910937C0070
:100B100000917500109176000819190920917A004A
:100B200030917B0036952795020F131F10F40FEFBD
:100B30001FEF00937A0010937B0029C020917A0068
:100B400030917B003901B4E08B2EB2E09B2E343023
:100B500010F08A949A94383010F08A949A9476948B
:100B600067948A94E1F726193709992021F01695A0
:100B700007959A94E1F7200F311F20937A00309364
:100B80007B0028F43FEF30937A0030937B003230C3
:100B900008F4706471FF02C0B3E00DC0B091C600EC
:100BA00000917100023838F0B395003A08F0B3951F
:100BB000B63008F0B5E09B2EB4E08B2E10917B0090
:100BC00000917A0024E0169507952A95E1F7081917
:100BD000120928F0B02FB250B12FB20910F402E080
:100BE00010E0980126C020917A0030917B003901F5
:100BF00076946794669466946694261932090695ED
:100C00000695200F321D20937A0030937B003230FE
:100C100008F07F7B04E03695279536952795269535
:100C20002695201B10F0223008F422E089019090D4
:100C3000C60060FDFECFE0908C00F0908D006160FA
:100C4000B9B7B061B9BF380176FD44C076946794F6
:100C500000938C0010938D00B92DB330E1F0B0FDFE
:100C600004C0060D171D930106C0000F111F02508E
:100C7000120922E030E0B92DB33068F020938E00E5
:100C800030938F00009388001093890060928A004F
:100C900070928B003DC000938E0010938F002093C4
:100CA00088003093890060928A0070928B0071FFF7
:100CB00010C0B0916D00B33060F000918F001091C2
:100CC0007C001595010F28F022F020928E000093F1
:100CD0008F001EC0669400938C00B92DB33091F044
:100CE000B0FD03C0060D262D03C0000F025022E008
:100CF000B92DB33038F020938E00009388006092B5
:100D00008A0006C000938E002093880060928A00BB
:100D100000917D0002FD0350013031F495FD0FC0BC
:100D2000B0B7B77FB0BF11C0023039F4B0B7B86008
:100D3000B0BFB4E0B06CB7B908C095FDF1CFB0B7A3
:100D4000B860B0BFB5E0B06CB7B90091A400000FB7
:100D500010F4BBE60B270093A40060FDFECFB2E0C9
:100D6000B0936E006160B9B7B061B9BFB72FB6700C
:100D7000A1F020917A0030917B0036952795F89468
:100D80000CB51DB5020F131F1BBD0ABD6160B0E19C
:100D9000B8BFB9B7B061B9BF7894089560612092C7
:100DA0007E0020E067FD20E206C0606120927E00A8
:100DB00020E267FD20E0789401E076FD11C0B72FB6
:100DC000B67009F06F7EB0917B00B55048F002E03C
:100DD000B55020F003E0B55008F006E071FD0AE0E0
:100DE00060FD12C0B0917E00BB2371F071FF08C09E
:100DF000B0916D00B33020F0B0916E00BA9519F447
:100E0000789470615EC0AEDF789400000000F894C2
:100E100076FD16C010917B00173008F017E0B5E0A2
:100E20001B0F72FD10E183FF110F62FF110F71FDA7
:100E300012E8B4B56090A100B61990F2B10B80F23F
:100E4000B0B71B2FB77FB0BFB8B1B0B713FDB86054
:100E5000B0BFB0917E00B395B0937E00B8B176FD7F
:100E600006C0B1E071FDB2E0BA95F1F7B8B1B07269
:100E7000B21709F01BC071FF05C003950A3008F0D6
:100E80000395AECF64FF97CF6F7E3CB56DB4709085
:100E90007A0080907B00370D681C6BBC3ABD6160A6
:100EA000B0E1B8BFB9B7B061B9BF85CFB0916D003F
:100EB000B23008F480CF64FD7ECF0A9509F090CF60
:100EC0007F7E20918E0030918F00F894B0E1B8BF02
:100ED0000CB51DB5020F131F1BBD0ABDE0908800A5
:100EE000F09089006160B9B7B061B9BF7894B72F4D
:100EF000B67039F0B0916D0072FFB395B0936D008C
:100F000009C074FF07C067FD05C064FD03C0BF9141
:100F1000BF91E5C4089500E063FF03C064FF01C012
:100F200001E0F89410917100B7E01B9F212D102D66
:100F30007894200F26951795269517952695179541
:100F400010937100183718F4B8E7B093710000914E
:100F50007100B09172000B1720F06062C098C198C8
:100F6000C29860FDFECFE0908A00F0908B00616037
:100F7000B9B7B061B9BF0895B2E095FD07C0F89464
:100F8000B0937D009498939A7894E5C0F894B093C8
:100F90007D009498959A7894DEC0B3E082FF24C0D7
:100FA00095FD11C002E0F894B0937D00E6E8F0E012
:100FB0000093B300C298959862FF02C0C19A01C025
:100FC000949A7894C8C002E0F894B0937D00E6E863
:100FD000F0E00093B300C098939862FF02C0C19AFA
:100FE00001C0949A7894B7C095FD0BC0F894B09363
:100FF0007D00E0E7F0E0C29862FF01C0C19A7894FA
:10100000AAC0F894B0937D00E0E7F0E0C09862FFDA
:1010100001C0C19A78949FC0B4E095FD07C0F894D0
:10102000B0937D009398959A789495C0F894B09376
:101030007D009598939A78948EC0B5E082FF24C085
:1010400095FD11C001E0F894B0937D00ECE7F0E06D
:101050000093B300C198949862FF02C0C09A01C087
:10106000939A789478C004E0F894B0937D00E0E916
:10107000F0E00093B300C198949862FF02C0C29A56
:1010800001C0959A789467C095FD0BC0F894B09311
:101090007D00EAE6F0E0C19862FF01C0C09A789452
:1010A0005AC0F894B0937D00E6E7F0E0C19862FF83
:1010B00001C0C29A78944FC0B6E095FD07C0F8947D
:1010C000B0937D009598949A789445C0F894B09325
:1010D0007D009398949A78943EC0B1E082FF24C03A
:1010E00095FD11C004E0F894B0937D00E0E9F0E0D4
:1010F0000093B300C098939862FF02C0C29A01C0E7
:10110000959A789428C001E0F894B0937D00ECE7BC
:10111000F0E00093B300C298959862FF02C0C09AB5
:1011200001C0939A789417C095FD0BC0F894B093C2
:101130007D00E6E7F0E0C09862FF01C0C29A7894B3
:101140000AC0F894B0937D00EAE6F0E0C29862FF2E
:1011500001C0C09A78946F7D089529E630E0F901C6
:101160002092B300C098C198C2989398949895988B
:101170006B7F0895A4EBB0E009E00D9309E00D93B7
:1011800004E00D930FEF0D9303E00D930FEF0D931C
:1011900009E00D9303E00D9301E00D9301E00D9341
:1011A000A0ECB0E001E00D930FEF0D930D930D93C4
:1011B0000D930D9303E00D930FEF0D930FEF0D9330
:1011C0000D9305E20D9300ED0D9308E20D9300E5FC
:1011D0000D9304E00D930FEF0D9302E00D9300E0EB
:1011E0000D930AE70D930FEF0D9300E00D9301E0CF
:1011F0000D9300E00D9303E00D9308952091BB0043
:101200008B7F233009F48460B091BC00B33019F0B7
:101210009F7DB1FD90629F7BB091BD00B1FD906458
:10122000223011F0886001C0877F08950A95E00F91
:10123000F21DB4910895ECE1F0E00091B400F6DF06
:10124000B093D800ECE1F0E00091B500EFDFB0938F
:10125000D900EAE2F0E00091BA00E8DFB093DA00EA
:10126000B091D0000FEF1CE0B23011F400EA1AE0A8
:10127000B33011F402E815E000937200109373008C
:10128000E8E3F0E00091D700D1DFB093A200089529
:1012900008952091CA003091CB00B091BC00B330CA
:1012A00009F43E5097FF02C020E03FEFB32FB21B7E
:1012B0006B2EB25810F4B2E86B2E00E00395609EDE
:1012C000B12DBD57D8F30093AE0008959068E1DFCB
:1012D000B9D920E030E0B0E16B2EB0D9B0919700E1
:1012E0002B0F321D6A94C9F7B4E036952795BA954D
:1012F000E1F7822E9F77CDDF0895F894E3E0F0E0E8
:10130000B9E0B7BFB491B078C1F3F894A895B1B57E
:10131000B861B1BDB0E0B1BDB4E0BEBFBFE5BDBF17
:101320001CDFB0E0B8BBB7E1B7BBB0E0B5BBB0E025
:10133000B4BBB0E0B2BBB8E3B1BB2224A0E0B0E0E4
:101340002D92AA31E9F7A0E6B0E00FEF2D920A95B1
:10135000E9F7B1E0B093A4000DDFF5D2B0E0B06CD6
:10136000B7B9B6B1B460B068B6B90091CC0000931B
:10137000AF00B1E0B0936A00F89468D972D962D92D
:1013800073D960D974D95ED9F8940AEF1AEFA0B373
:1013900096FDA095A2FF1FC01A95C9F70A95B1F74F
:1013A000E0E0FCE1B591B43E39F4B591B03E21F4F2
:1013B000B591BF3F09F40CC0E0E0F395F395B5910A
:1013C000B83F49F4B591B43931F4B591BA3A19F44A
:1013D000EE27F695099412DF2EDF5ADF5ADF0091CF
:1013E000CC000093AF00B9DEB2E0B3BFB2E0BEBD47
:1013F000B2E0B5BDB1E5B8BFB9BFB0B70B2FB77F8D
:10140000B0BFB8B1B0B703FDB860B0BF15D978941C
:10141000D5DAB3E096FDB2E0B5BFB0E4BBBFBB2701
:10142000B064BABF8D7F12D9626033E02CE0B09116
:101430009600BB2321F42CE03A9509F4A5CF02D9FC
:1014400080FFA2CF8E7FB0919700B23078F3B92F92
:10145000BF710091990000939800B0939900B01764
:1014600029F72A9521F76D7FB3E096FDB2E0B5BF6D
:10147000BB27B064BABF8D7FB091D600BB2321F4E7
:101480008062B92FB0709B2F8F7B20926700DCD8D1
:1014900085FF05C0B0916700BA3008F08064CED8EF
:1014A00002E085FF01C000E0B0919700B017B8F3EB
:1014B000F894D7D8D6D8D5D87894C8D820928700B1
:1014C000B091BC00B33009F474C0B8D8B091C0007A
:1014D000B13008F46EC0B0916A00B13008F469C050
:1014E00085FD18C0B0919700BF3F08F462C0F89422
:1014F000C1D87894A9D8B0919700B130C0F7F894CA
:10150000B0D89ED8AED878949FD8B0919700BF3FFE
:10151000B0F3DAC2B3E09B2E9068F894BADE789408
:1015200093D8F8949F77B5DE80909700B09197009C
:10153000BF37789408F445C07FD8F8949BD8789446
:101540009A9451F7C3DEB82DB550B093CB007ED836
:10155000F89426D28CD27894BAE09B2E9068F894B6
:1015600098DE789471D8F8949F7793DE80909700F6
:10157000B0919700BF37789478F75ED8F89471D817
:101580005FD86FD878949A9449F7A0DEB82DBB5FE6
:10159000B093CA005BD8F89403D278D2789454D828
:1015A000F89477DE7894B0919700BF3F08F498CF15
:1015B0008BC200919700B09187000B1710F0009339
:1015C000870042D801E0B091BC00B35009F405E0B7
:1015D000B0919700B01708F073CFF8944BD84AD861
:1015E00049D8789433D820926A0020926B002092D8
:1015F0006C00B0916B00B395B0936B00BF3F69F581
:10160000B0916C00B395B0936C00B091CE0009E13D
:10161000BA9559F002E3BA9541F00DE7BA9529F071
:101620000AEFBA9511F020926C00B0916C00B017DF
:10163000A0F0B0916C00BA95B0936C00B4EBB0938D
:101640006B00B091CD00B093AF00F89413D87894AC
:10165000B091CC00B093AF00F7D7F2D7B09168004B
:10166000BB2319F485FF01C08FCE01E085FD01C0C9
:1016700006E0B0919700B01708F4BBCFB091BC0062
:10168000B35009F0E1D7B0916800BB2309F47CCED8
:10169000F89463DD20926100209262002092630042
:1016A000522C209264002092A3007894B091B9004B
:1016B000BB0FB093A00020927F0020928000209268
:1016C000810020928200209283002092AC0060E092
:1016D00070E020927100B8E0B093AC007860ACD7B5
:1016E000B0E073FDB1E0B06CB7B9B6B1B068B0644A
:1016F000B6B9B6B1B6FDFDCF04B115B1B6B1BF777D
:10170000B6B9112309F00FEF0093AD0059D9B8E035
:10171000B093AC0078608090BB00B2E0B093BB00A7
:101720006DDD8092BB00F894BFEFB0939C00A7D909
:10173000B0916100B0939C00B0939D00B0939E0067
:101740007894B1E0B0936100B09363005B2EB093E6
:101750006400B093A600B0919B00B093A500B09137
:10176000BC00B33019F49F7D87FD90627160726098
:1017700020926D00A1DCB1DC9BD9A0D999D99ED96A
:1017800097D906C0F8943ADD78942092AC00777F20
:101790000CDBE7D7C0DBF0DB91D900DB66FD1AD8A4
:1017A00076FFCCD876FDFAD8B6DBF7DB87D9FDDA41
:1017B00066FD2CD8B0DB30DC81D9F0DA66FD60D86C
:1017C000AADB3BDC7BD9F1DA66FD8AD8A4DB74DCCA
:1017D00075D9E4DAB0E073FDB1E0B06CB7B9B6B179
:1017E000B068B064B6B997DB78DC68D9E9D871FF26
:1017F00026C067FD24C0B0919F00B0939C00B093B9
:101800009D00B0919B00B093A500B1E0B093A600FD
:1018100018E12CE0B0916D00B11758F07D7F746035
:1018200020936F00B0919F00B0939C00B0939E00F6
:1018300006C0B0919700B13008F0AACF5AC072FF2D
:1018400010C067FD0EC0B0916F00BA9511F47B7F98
:1018500099CFB0936F00B0919700B13008F098CF56
:1018600048C020927000B0919A000AEFB01708F0BB
:1018700040C085FF04C0B0916800BB23D1F1B09196
:10188000BC00B33081F495FD03C087FD04C00BC0DC
:1018900087FF01C008C067FD06C06068B0919F0067
:1018A000B0939C008ACF00EF67FF05C0B0919F0006
:1018B000B0939C0000E2B0917B00B01708F468CFB1
:1018C00067FF17C06F779F7D87FD90627460B2E1FC
:1018D000B0936F00B0919F00B0939C0059CFB0912E
:1018E0007000B395B0937000B0919700BB2309F0DE
:1018F00002C020927000F89430DC8090BB00B2E00F
:10190000B093BB007BDC8092BB00209261002092F0
:10191000620020926300522C209264002092A0006A
:101920007E7F789489D619DCB0E0B06CB7B9B6B1D7
:10193000B460B068B6B985FF05C0B0917000B5302D
:1019400008F022CD52CEEDE0F0E023D0053509F0CD
:101950001BC0EEE0F0E01DD00A3A09F015C03AE0F5
:10196000A4EBB0E0E3E0F0E014D00D9331963A95AB
:10197000D9F738E1A0ECB0E0EFE0F0E00AD00D9349
:1019800031963A95D9F702C0F5DB0AD0E7E2F0E0EC
:101990000895E199FECFEEBBFFBBE09A0DB3089529
:1019A0001ED03AE0A4EBB0E0E3E0F0E00D910FD000
:1019B00031963A95D9F738E1A0ECB0E0EFE0F0E0ED
:1019C0000D9105D031963A95D9F712D00895E19945
:1019D000FECF0DBBEEBBFFBBE29AE19A0895EDE0AE
:1019E000F0E00FEFF4DFEEE0F0E00FEFF0DF08954E
:1019F000EDE0F0E005E5EBDFEEE0F0E00AEAE7DF3E
:101A000008953091B0000091B100313011F400938D
:101A1000B400323011F40093B500333011F4009368
:101A2000B600343011F40093B800353011F400934F
:101A3000BA00363011F40093C600373011F4009329
:101A4000BB00383011F40093D700393011F4009303
:101A5000D0003A3011F40093BC003B3011F40093F5
:101A6000BD00089525E0F2D52A95E9F70895F9D546
:101A7000FBD5FDD5FFD5E4D5F4D5F6D5F8D5FAD507
:101A8000DFD5EFD5F1D5F3D5F5D50895F3D5EFD55D
:101A9000EBD5E7D5D5D5EED5EAD5E6D5E2D5D0D587
:101AA000E9D5E5D5E1D5DDD508958090B0009090D9
:101AB000B100D7D5D6D5D5D5C3D58A94D1F7DAD547
:101AC000BFD59A94E1F70895F894D1DF7894CADFEE
:101AD000C9DFB1E0B093B000B1E0B093B1002092A3
:101AE000B200F894E2DF7894B5E06B2E7090970026
:101AF000ADD5B09197007B16C9F7B13018F0BF3F54
:101B000040F107C07EDFF8944BDFB1DFB8E0B1BD34
:101B1000A9DF6A9459F7B091B200B395B093B200BF
:101B2000B33008F4DECF9EDFB091B100B395B0932F
:101B3000B100F894B091B000BA95EEE3F0E0EB0F8D
:101B4000F21D049178940395B091B100B01708F498
:101B5000C6CF88DF87DFB091B000B395B093B000F7
:101B6000B091B000BC3008F4B7CF04DBF89418DFB4
:081B7000B8E0B1BD77DFC1CB85
:00000001FF
